:100000000C9415050C94B9070C9492070C94E40910
:100010000C94E4090C94E4090C94260E0C943D0510
:100020000C943D050C943D050C943D050C943D0548
:100030000C943D050C94C60D0C943D050C943D05A7
:100040000C94E4170C943D050C9400090C94DA0808
:100050000C943D050C943D050C943D050C943D0518
:100060000C943D050C943D05451F481F4B1F4E1F2A
:10007000511F541F571FD021D321D621D921DC2154
:10008000DF21E221BE22C122C422C722CA22CD2200
:10009000D02242657374206361702E00204361702A
:1000A00061636974793A004265737420736574748E
:1000B000696E673A00092067697665732066726524
:1000C0007175656E63793A200074756E6520616E96
:1000D00074656E6E6120746F206361706163697412
:1000E0006F722000417272617920636C6561726584
:1000F000642E2E2E2E002E00436C656172206172DC
:100100007261792E2E2E2E00536574757020656EE7
:1001100074657265642E2E2E00436865636B2066DD
:100120006F72207365747570005479706520475341
:1001300020746F20656E7465722073657475703AF3
:100140000057726974696E672064656661756C74C6
:10015000732E2E2E2E005374617274206469737096
:100160006C617900626567696E6E696E6720626FA7
:100170006F742070726F6365647572652E2E2E2EFB
:10018000002E00506C6179696E6720576974682091
:10019000467573696F6E3A20415333393335204CBD
:1001A000696768746E696E672053656E736F722C31
:1001B0002053454E2D33393030312D5230312020EF
:1001C000760041736C6565700041542B47534C5069
:1001D0003D00427574746F6E207072657373656450
:1001E0003A00446973706C61793A005361747572B6
:1001F000646179004672696461790054687572734C
:10020000646179005765646E657364617900547543
:100210006573646179004D6F6E6461790053756E2A
:100220006461790020746F6F2068696768004E6FA1
:10023000697365206C6576656C004E6F6973652027
:100240006C6576656C20746F6F2068696768002044
:1002500020646574656374656400446973747572C1
:1002600062657200446973747572626572206465B8
:1002700074656374656400204B4D00204469737499
:100280003A003A003A002000204B4D0020204469FB
:1002900073742E20004C696768746E696E67002065
:1002A0006B696C6F6D6574657273004C6967687417
:1002B0006E696E67206465746563746564212044AB
:1002C000697374616E636520746F20737472696BF7
:1002D000653A2000206E6F742065787065637465E0
:1002E000640020736F7572636520726573756C743A
:1002F00000696E7465727275707400696E746572EF
:100300007275707420736F75726365207265737592
:100310006C74206E6F74206578706563746564001A
:100320002F0050756C7365733A004461792020206A
:100330003A00486F757220203A004D696E757465F9
:100340003A0053746174733A002A2A2A0053617484
:1003500000467269005468750057656400547565FD
:10036000004D6F6E0053756E004B4D0020004869C4
:1003700073746F72793A004461792020203A004802
:100380006F757220203A004D696E7574653A0020D1
:100390002A00536174757264617900467269646100
:1003A00079005468757273646179005765646E658D
:1003B000736461790054756573646179004D6F6E83
:1003C0006461790053756E646179002020202020DB
:1003D00020202A00202020202A00202A002020423D
:1003E0007574746F6E74696D653A004573636170FE
:1003F00065642066726F6D206C6F6F703A002E001E
:10040000204465746563746F7220760020204C6907
:100410006768746E696E670020202050493452412D
:100420005A0044697361626C656400456E61626C78
:10043000656400446973743A00496E646F6F727347
:10044000004F7574646F6F72004D6F64653A0043BE
:10045000616C6C3A004E6F20636F6E6E65637469F9
:100460006F6E002A0020204842433D00496E666FAF
:100470003A00293A00436F6E747261737428002940
:100480003A0053637265656E2031202830202D209C
:100490003329202800293A0054696D6520636F7262
:1004A00072656374696F6E202800293A004E6F6987
:1004B00073656C6576656C202831202D20382920E5
:1004C0002800293A0043617061636974792028002B
:1004D000293A0023426565706572202800293A2078
:1004E00000456E61626C65640044697361626C65AD
:1004F00064004469737475726265722028302F310C
:1005000029202800293A20004F7574646F6F727398
:1005100000496E646F6F727300496E646F6F72731F
:100520003D30206F72204F7574646F6F72733D3170
:10053000202800293A0043616C6C202800293A00E9
:1005400050617373776F7264202800293A00535307
:1005500049442028005761746368646F672072659E
:1005600063656976656420286D61782031302920C3
:100570000072656164790041544530004154004186
:10058000542B525354003C2D2D2D200041542B430D
:1005900049504D55583D3000222C220041542B43E8
:1005A000574A41503D220041542B43574D4F44453B
:1005B0003D310041542B43494653520041542B4393
:1005C00049505345525645523D300041542B434902
:1005D000504D55583D300041542B4349465352002D
:1005E0004661696C65643A2068617264776172651E
:1005F000207265736574004661696C65643A2073A6
:100600006F66747761726520726573657400466108
:10061000696C65643A20636F6E6E656374696E67BA
:10062000004661696C65643A204E6F204950206E27
:10063000756D6265720053657420746F2073696E06
:10064000676C6520636F6E6E656374206D6F6465A3
:10065000005365727665726D6F646520616C7265BA
:1006600061647920736574005365727665726D6F8D
:10067000646520736574004F4B0A436865636B695A
:100680006E6720495020616464722E2E2E00436FE5
:100690006E6E656374696E6720746F205769466972
:1006A0002E2E2E005365742054696D654F7574733A
:1006B0002E2E2E00536F66742072657365742E2E75
:1006C0002E00486172642072657365742E2E2E00B0
:1006D00020485454502F312E310D0A486F73743A0C
:1006E000206F6E776565722E70693472617A2E6E36
:1006F0006C002644697374616E63653D0026496E23
:1007000074547970653D00474554202F4164644519
:1007100076656E742E7068703F43616C6C736967A8
:100720006E3D006F6E776565722E70693472617A06
:100730002E6E6C00474554202F74696D652E7068CD
:100740007020485454502F312E310D0A486F737465
:100750003A206F6E776565722E70693472617A2EF9
:100760006E6C006F6E776565722E70693472617A97
:100770002E6E6C002D2D2D3E20000000000000008C
:10078000005F00000007000700147F147F14242A74
:100790007F2A12231308646236495522500005034C
:1007A0000000001C2241000041221C0014083E08E9
:1007B0001408083E0808005030000008080808081F
:1007C000006060000020100804023E5149453E00D0
:1007D000427F400042615149462141454B31181446
:1007E000127F1027454545393C4A49493001710976
:1007F00005033649494936064949291E003636005F
:100800000000563600000814224100141414141479
:1008100000412214080201510906324979413E7E05
:100820001111117E7F494949363E414141227F41A4
:1008300041221C7F494949417F090909013E41493B
:10084000497A7F0808087F00417F41002040413FEE
:10085000017F081422417F404040407F020C027F0C
:100860007F0408107F3E4141413E7F090909063E51
:100870004151215E7F091929464649494931010103
:100880007F01013F4040403F1F2040201F3F403834
:10089000403F631408146307087008076151494515
:1008A00043007F41410002040810200041417F00C5
:1008B00004020102044040404040000102040020C4
:1008C000545454787F48444438384444442038448D
:1008D00044487F3854545418087E0901020C52527F
:1008E000523E7F0804047800447D40002040443D8F
:1008F000007F1028440000417F40007C04180478E9
:100900007C0804047838444444387C1414140808DF
:100910001414187C7C080404084854545420043FE0
:100920004440203C4040207C1C2040201C3C403067
:10093000403C44281028440C5050503C4464544CD3
:1009400044000836410000007F00000041360800E6
:1009500010080810080000000000556E6C696E6BEE
:100960000D0A0041542B434950434C4F534500411D
:10097000542B43495053454E443D003C2D2D2D20D2
:10098000004F4B0D0A00476F742049503A004461F4
:1009900074652654696D6520666F756E64002B2B37
:1009A0002B2B2B2B002D2D2D2D2D2D00000000008D
:1009B000250028002B00000000002300260029004D
:1009C00004040404040404040202020202020303F5
:1009D00003030303010204081020408001020408FD
:1009E000102001020408102000000000240027004D
:1009F0002A000000000800020100000304070000B4
:100A0000000000000000456E657267793A00222CF4
:100A10000041542B43495053544152543D225443B6
:100A200050222C22000036232C2311241FBECFEF8E
:100A3000D8E0DEBFCDBF25E0A6E9B2E001C01D923F
:100A4000A13AB207E1F712E0A0E0B1E0EEE6FAE485
:100A500002C005900D92A639B107D9F715E0C4E19F
:100A6000D5E004C02197FE010E94DD24C331D107E7
:100A7000C9F70E942E180C942A250C9400000895A2
:100A8000CF92DF92EF92FF920F931F93CF93DF935A
:100A90006C017A018B01C0E0D0E0CE15DF0589F052
:100AA000D8016D918D01D601ED91FC910190F081FD
:100AB000E02DC6010995892B11F47E0102C0219613
:100AC000ECCFC701DF91CF911F910F91FF90EF9075
:100AD000DF90CF900895FC01538D448D252F30E099
:100AE000842F90E0821B930B541710F0CF9608953B
:100AF00001970895FC01918D828D981761F0828D88
:100B0000DF01A80FB11D5D968C91928D9F5F9F7341
:100B1000928F90E008958FEF9FEF0895FC01918DE3
:100B2000828D981731F0828DE80FF11D858D90E050
:100B300008958FEF9FEF0895FC01918D228D892FED
:100B400090E0805C9F4F821B91098F7399270895D5
:100B50008AE694E00E949C0521E0892B09F420E0BC
:100B6000822F0895FC01848DDF01A80FB11DA35AC7
:100B7000BF4F2C91848D90E001968F739927848FBD
:100B8000A689B7892C93A089B1898C9180648C93B4
:100B9000938D848D981306C00288F389E02D80819F
:100BA0008F7D80830895EF92FF920F931F93CF93D1
:100BB000DF93EC0181E0888F9B8D8C8D981305C0AD
:100BC000E889F989808185FD24C0F62E0B8D10E01F
:100BD0000F5F1F4F0F731127E02E8C8DE8120CC092
:100BE0000FB607FCFACFE889F989808185FFF5CF38
:100BF000CE010E94B205F1CF8B8DFE01E80FF11DF1
:100C0000E35AFF4FF0820B8FEA89FB898081806273
:100C100007C0EE89FF896083E889F9898081806453
:100C2000808381E090E0DF91CF911F910F91FF9041
:100C3000EF900895CF93DF93EC01888D8823C9F05E
:100C4000EA89FB89808185FD05C0A889B9898C91D5
:100C500086FD0FC00FB607FCF5CF808185FFF2CF70
:100C6000A889B9898C9185FFEDCFCE010E94B2058C
:100C7000E7CFDF91CF91089580E090E0892B29F0B4
:100C80000E94A80581110C940000089520919802FB
:100C9000309199022817390771F49091960280914A
:100CA0009702981741F0E0919602F0E0ED58FC4F62
:100CB000808190E008958FEF9FEF089508951F932E
:100CC000CF93DF93DC015C962D913C915D972115CC
:100CD000310539F481E090E013969C938E9312973E
:100CE0003DC05196ED91FC91529750969C91509732
:100CF000892F80951FB75E964C915E9741FB7727B1
:100D000070F941FD6095F8944081772311F0492BEB
:100D100001C048234083E9012197F1F748E0508161
:100D200060FF02C0592B01C058235083E90121976D
:100D3000F1F76695415099F7772321F09081892347
:100D4000808303C08081982B90831FBF5C968D9118
:100D50009C915D970197F1F721E030E0C901DF91A7
:100D6000CF911F91089520919802309199022817F0
:100D7000390771F4809197022091960290E0805C8F
:100D80009F4F821B910960E470E00E94A7240895A0
:100D900080E090E008952091980230919902281700
:100DA0003907B9F49091960280919702981789F0CB
:100DB000E0919602F0E0ED58FC4F80812091960280
:100DC00030E02F5F3F4F2F7333272093960290E040
:100DD00008958FEF9FEF0895089580E090E00895C3
:100DE00081E080939E020895CF93DF93CAE0D0E024
:100DF0008AE694E00E949C05181619062CF48AE6EF
:100E000094E00E947A05F4CF219791F7DF91CF917A
:100E10000895FF920F931F93CF93DF930E94F406E0
:100E20001092C80300E010E0F12CD0E0C0E0DD300B
:100E300069F18AE694E00E949C0518161906BCF731
:100E40008AE694E00E947A05D82F80ED8D0F8A30D3
:100E500098F4F801E853FC4FD0830F5F1F4F6D2FBC
:100E60008AE694E00E94D305CC0F8C2F880F880F60
:100E7000C80FC053CD0FDBCFDD32C9F66DE28AE675
:100E800094E00E94D305FF24F394D3CFF801E853F4
:100E9000FC4F1082F110C1950E94F4068C2FDF9157
:100EA000CF911F910F91FF900895EF92FF920F93B2
:100EB0001F93CF93DF937C010E94F4061092C80326
:100EC000C0E0D0E08E0108531C4FF80180818D30C6
:100ED00051F4F8011082DF91CF911F910F91FF9093
:100EE000EF900C94F406CE15DF059CF78AE694E0AB
:100EF0000E949C051816190644F78AE694E00E94A1
:100F00007A05682FF80180838D3011F08A3011F452
:100F1000219704C08AE694E00E94D3052196D2CF9F
:100F20000E94F7241F920F920FB60F9211242F9355
:100F30003F934F935F936F937F938F939F93AF9361
:100F4000BF93EF93FF93E0910501F091060109959E
:100F5000FF91EF91BF91AF919F918F917F916F9191
:100F60005F914F913F912F910F900FBE0F901F9067
:100F700018951F920F920FB60F9211242F933F9343
:100F80004F935F936F937F938F939F93AF93BF9391
:100F9000EF93FF93E0910301F09104010995FF9114
:100FA000EF91BF91AF919F918F917F916F915F91E1
:100FB0004F913F912F910F900FBE0F901F9018955A
:100FC0000F931F93CF93DF93EC010E94D81768878C
:100FD00079878A879B87E881F9810284F385E02DF0
:100FE000CE01099597FF17C00E94D817088519856B
:100FF0002A853B85DC01CB01801B910BA20BB30B37
:101000000C811D812E813F8180179107A207B307B4
:1010100010F38FEF9FEFDF91CF911F910F91089504
:10102000DC01ED91FC910190F081E02D0994EF92AB
:10103000FF920F931F93CF93DF938C017B01C0E04E
:10104000D0E0F701EC0FFD1F6491662361F0D80139
:10105000ED91FC910190F081E02DC8010995892B5B
:1010600011F02196EECFCE01DF91CF911F910F911C
:10107000FF90EF9008951F93CF93DF93EC01162F0D
:101080008E819F81009799F02B8D211106C064E716
:1010900077E00E94170881E08B8F8E819F81DC01B1
:1010A000ED91FC910190F081E02D612F09958C81EB
:1010B0009D81DC01ED91FC910190F081E02D612F8B
:1010C000DF91CF911F9109946115710579F0FB01B2
:1010D00001900020E9F73197AF01461B570BDC0167
:1010E000ED91FC910280F381E02D099480E090E085
:1010F00008954F925F926F927F92EF92FF920F93BB
:101100001F93CF93DF93CDB7DEB7A1970FB6F894B7
:10111000DEBF0FBECDBF7C01FA01CB0119A2223088
:1011200008F42AE08E010F5D1F4F422E512C612CD6
:10113000712CBF01A30192010E94BB24F901CA01D5
:10114000015011096A3014F4605D01C0695CD80176
:101150006C93232B242B252B61F7B801C7010E9428
:101160006408A1960FB6F894DEBF0FBECDBFDF9125
:10117000CF911F910F91FF90EF907F906F905F90B4
:101180004F9008956CE072E00C9464080F931F93E5
:10119000CF93DF93EC010E9417088C01CE010E94CF
:1011A000C208800F911FDF91CF911F910F91089579
:1011B0000C9464081F920F920FB60F9211242F9374
:1011C0003F934F935F936F937F938F939F93AF93CF
:1011D000BF93EF93FF938AE694E00E94B205FF91DC
:1011E000EF91BF91AF919F918F917F916F915F919F
:1011F0004F913F912F910F900FBE0F901F90189518
:101200001F920F920FB60F9211242F938F939F93DB
:10121000EF93FF93E0917A04F0917B048081E09159
:101220008004F091810482FD12C09081809183043A
:101230008F5F8F7320918404821751F0E0918304B3
:10124000F0E0E659FB4F958F8093830401C08081C5
:10125000FF91EF919F918F912F910F900FBE0F9063
:101260001F901895CF92DF92EF92FF920F931F93EA
:10127000CF93DF93EC01E42E8E810E941A1760E079
:1012800088850E941A17DC80CD8007E010E0F12CE1
:10129000B701002E02C0759567950A94E2F7617058
:1012A00077278C2D0E941A1761E08D2D0E941A1746
:1012B00060E08D2D0E941A170150110948F761E076
:1012C0008885DF91CF911F910F91FF90EF90DF9074
:1012D000CF900C941A17CF92DF92EF92FF920F9358
:1012E0001F93CF93DF9300D000D01F92CDB7DEB70E
:1012F00067FD57C07C01862F90E0603260F08097D8
:1013000025E0289FB001299F700D11246658784F61
:1013100045E050E00FC0FC013796EE0FFF1FEE0DC9
:10132000FF1D008111810115110559F445E050E0C0
:101330006AE777E0CE0101960E9464248E010F5F78
:101340001F4F680185E0C80ED11CF80141918F0143
:1013500061E0C7010E9432090C151D05B1F740E09C
:1013600061E0C7010E943209F701848590E006968A
:10137000628570E00E94A7248487811115C02585AD
:1013800030E02F5F3F4F938569E3969F612D1124D5
:10139000669570E06F5F7F4FC9010E94A724858723
:1013A00003C080E090E002C081E090E00F900F90D9
:1013B0000F900F900F90DF91CF911F910F91FF90A1
:1013C000EF90DF90CF9008951F920F920FB60F927B
:1013D00011242F933F934F935F936F937F938F933A
:1013E0009F93AF93BF93EF93FF93E0919802F09197
:1013F0009902309709F451C0968DA685B7858585E9
:1014000091FF04C09C91892329F447C09C918923B2
:1014100009F043C0A389B4899C918589809589236B
:101420008C93868997890197F1F7608D718DA685D8
:10143000B785558538E020E0CB010197F1F7822F81
:1014400090E095958795282F4C91452309F02068C9
:10145000315091F7868D81FD20958091970290E023
:1014600001968F73992730919602381749F0A09111
:101470009702B0E0AD58BC4F2C938093970203C005
:10148000868D8160868F828D938D0197F1F7A38978
:10149000B4899C918589892B8C93FF91EF91BF91A1
:1014A000AF919F918F917F916F915F914F913F91FC
:1014B0002F910F900FBE0F901F901895E0919802FA
:1014C000F0919902E817F90769F4A389B4899C910E
:1014D0008589809589238C931092990210929802A5
:1014E00081E0089580E0089560E08DE00E941A1781
:1014F00040E260E082E495E00C9432090C9476249A
:101500004F925F926F927F928F929F92AF92BF9213
:10151000CF92DF92EF92FF920F931F93CF93DF93BF
:10152000CDB7DEB7DA950FB6F894DEBF0FBECDBFEC
:1015300010929A0210929F0262EC76E08AE694E0A2
:101540000E94C60880911F0587FF24C064EB76E0E7
:101550008AE694E00E94C608C0900F05D09010055E
:10156000E0901105F09012058091130590911405FB
:10157000A0911505B09116050097A105B10509F4D4
:101580007FC080930F0590931005A0931105B09331
:10159000120576C0C0900F05D0901005E09011059F
:1015A000F0901205409113055091140560911505B6
:1015B00070911605411551056105710541F0409383
:1015C0000F0550931005609311057093120548E8BC
:1015D00053E160E070E0409313055093140560936D
:1015E00015057093160548E95AE360E070E04093F2
:1015F0001705509318056093190570931A0560E05C
:101600000E941A1761E080911F050E944A1764E644
:1016100070E080E090E00E94861760E080911F05F6
:101620000E944A17C114D104E104F10441F0C092B0
:101630000F05D0921005E0921105F092120588E88E
:1016400093E1A0E0B0E08093130590931405A0937C
:101650001505B093160588E99AE3A0E0B0E0809301
:10166000170590931805A0931905B0931A0581E703
:1016700095E00E94B114811169CF60EE75E0BDC1A3
:1016800038E8832E33E1932EA12CB12C80921305E0
:1016900090921405A0921505B092160548E9442EC3
:1016A0004AE3542E612C712C409217055092180574
:1016B0006092190570921A056FE775E087E095E072
:1016C0000E94C60880E090E00E94B1148823D1F007
:1016D0006CE775E087E095E00E94C60880E090E046
:1016E0000E94B11467E775E087E095E00E94C608A4
:1016F00080E090E00E94B114C114D104E104F1042F
:1017000081F007C0C114D104E104F10409F44EC111
:1017100080E0C0920F05D0921005E0921105F09282
:10172000120598E8892E93E1992EA12CB12C809274
:10173000130590921405A0921505B092160528E99C
:10174000C22E2AE3D22EE12CF12CC0921705D092A2
:101750001805E0921905F0921A05882309F436C19C
:1017600064EA76E08AE694E00E94C60888EE93E098
:10177000A0E0B0E080930F0590931005A0931105B1
:10178000B09312058092130590921405A09215054E
:10179000B0921605C0921705D0921805E09219056F
:1017A000F0921A056EE876E08AE694E00E94C60898
:1017B00080910D0590910E05009751F02091220522
:1017C000222331F066E875E00E9417081092220586
:1017D000A0900B05B0900C05CE0101967C0100E0B5
:1017E00010E06C01C5010E94E00797FD0BC08D3031
:1017F000910541F0D7018D937D010F5F1F4F0F3F82
:10180000110581F7F601E00FF11F108280910B05A1
:1018100090910C05DC01ED91FC910284F385E02DA3
:1018200009950A9799F767EA75E087E095E00E94C5
:10183000C60880E090E00E94B114882309F4B3C088
:101840006CE975E087E095E00E9417086DE071E0B3
:1018500087E095E00E94D80868E975E087E095E0A8
:101860000E9417086DE171E087E095E00E94D808BA
:1018700062E287E095E00E94100887E095E00E9410
:10188000C208C0900F05D0901005E0901105F090AF
:1018900012058091170590911805A0911905B09136
:1018A0001A050097A105B10541F080930F059093AB
:1018B0001005A0931105B093120588E893E1A0E00C
:1018C000B0E08093130590931405A0931505B09391
:1018D000160588E99AE3A0E0B0E08093170590939D
:1018E0001805A0931905B0931A0580E090E00E94B6
:1018F000B114C114D104E104F10441F0C0920F0508
:10190000D0921005E0921105F092120548E853E1DB
:1019100060E070E040931305509314056093150543
:101920007093160548E95AE360E070E040931705AC
:10193000509318056093190570931A05882399F13F
:101940006CE875E087E095E00E94C60880E090E0D2
:101950000E94B114882339F167E776E08AE694E0C3
:101960000E94C60863EB75E087E095E00E94C60818
:1019700080E090E00E94B114882391F081E0809390
:101980009A026CEB75E087E095E00E94C60880E063
:1019900090E00E94B1148823E1F068E676E01BC075
:1019A00061E276E02AC06EE076E027C080921305FF
:1019B00090921405A0921505B09216054092170555
:1019C000509218056092190570921A0567EF75E03C
:1019D00014C061E576E08AE694E00E94C6086BECEC
:1019E00075E087E095E00E94C60880E090E00E94E4
:1019F000B114882331F066E376E08AE694E00E9431
:101A0000C60880919A02882399F067ED75E083E219
:101A100095E00E94C6080E943F1303E010E0809109
:101A2000C703811102C00E942F0D01501109B9F79F
:101A3000D3950FB6F894DEBF0FBECDBFDF91CF9127
:101A40001F910F91FF90EF90DF90CF90BF90AF90DC
:101A50009F908F907F906F905F904F9008958091AE
:101A60009F0281110E94800A80919A02882321F1AD
:101A700083E697E00E94BF158823E1F00E943F13A0
:101A800084E390E00E944C158823A1F064E377E0A2
:101A900083E295E00E94C60883E295E00E94C208B6
:101AA00083E295E00E94C2080E943F130E943F1308
:101AB0000E943F130C94671508950F931F93CF93C3
:101AC000DF93082F162F80919F0281110E94800AB8
:101AD00080919A02882309F454C083E297E00E941F
:101AE000BF15882309F447C01A3018F0C0E6D0E0CB
:101AF00002C0CFE5D0E0BE018AE694E00E94DF118B
:101B0000CE010E944C158823B1F167E077E083E2B3
:101B100095E00E94170868E371E083E295E00E9477
:101B2000D8086DEF76E083E295E00E941708602FF9
:101B300083E295E00E94061262EF76E083E295E090
:101B40000E941708612F83E295E00E94061260ED63
:101B500076E083E295E00E94C60883E295E00E9469
:101B6000C20883E295E00E94C2080E943F130E94CF
:101B70003F130E943F13DF91CF911F910F910C945F
:101B80006715DF91CF911F910F9108951F920F92CA
:101B90000FB60F9211242F933F934F935F936F9340
:101BA0007F938F939F93AF93BF93EF93FF938EEEAB
:101BB00095E89093850080938400809172038F5FF5
:101BC0008A3718F48093720302C0109272038091D6
:101BD000720386958093C5038C3339F51092720396
:101BE0001092C5038091C6038F5F8093C6036FE098
:101BF00072E08AE694E00E94D8088091C6038C3394
:101C0000A1F41092C6038091C7038F5F883119F049
:101C10008093C7030AC01092C70380914B018F5F66
:101C2000883009F481E080934B01FF91EF91BF91DF
:101C3000AF919F918F917F916F915F914F913F9164
:101C40002F910F900FBE0F901F9018951F920F921B
:101C50000FB60F9211242F933F934F935F936F937F
:101C60007F938F939F93AF93BF93EF93FF93A89529
:101C700080919C0290919D02019690939D02809389
:101C80009C0265E575E08AE694E00E941708609181
:101C90009C0270919D028AE694E00E94DF1180917F
:101CA0009C0290919D020A9719F4E0E0F0E00995FA
:101CB000FF91EF91BF91AF919F918F917F916F9124
:101CC0005F914F913F912F910F900FBE0F901F90FA
:101CD00018950F931F93CF93DF9380E090E00E94BD
:101CE0007E0A90910C0189130EC00CE011E0C0E057
:101CF000D0E0CE010E947E0AF80181938F012196E7
:101D0000CF33D105B1F7DF91CF911F910F91089596
:101D10000F931F93CF93DF930CE011E0C0E0D0E06E
:101D2000F80161918F01CE010E947E242196CF336C
:101D3000D105B1F7DF91CF911F910F910895CF9306
:101D4000C82F6EE475E08AE694E00E9417086DE003
:101D500071E08AE694E00E94D8086BE475E08AE6B8
:101D600094E00E941708CC2381F08FE090E00E945D
:101D700055078091C803882341F010920D0168EC4B
:101D800073E08DE091E00E9405258AE694E00E94D0
:101D9000C20860E475E08AE694E00E9417086DE1ED
:101DA00071E08AE694E00E94D8086DE375E08AE667
:101DB00094E00E941708CC2381F08AE190E00E9411
:101DC00055078091C803882341F010921D0168ECEB
:101DD00073E08DE191E00E9405258AE694E00E947F
:101DE000C20866E375E08AE694E00E94170868E39B
:101DF00071E08AE694E00E94D80863E375E08AE621
:101E000094E00E941708CC2381F089E090E00E94C2
:101E100055078091C803882341F01092380168EC7F
:101E200073E088E391E00E9405258AE694E00E9431
:101E3000C20869E175E08AE694E00E941708809183
:101E40004201811103C061E175E002C068E075E004
:101E50008AE694E00E94170864E075E08AE694E060
:101E60000E941708CC2339F00E9409079091C803FB
:101E70009111809342018AE694E00E94C20862EFC9
:101E800074E08AE694E00E94170880914301811172
:101E900003C069EE74E002C061EE74E08AE694E08B
:101EA0000E9417086DED74E08AE694E00E9417081E
:101EB000CC2339F00E9409079091C80391118093B7
:101EC00043018AE694E00E94C20863ED74E08AE66A
:101ED00094E00E941708609144018AE694E00E9411
:101EE000061260ED74E08AE694E00E941708CC23A5
:101EF00039F00E9409079091C80391118093440121
:101F00008AE694E00E94C20865EC74E08AE694E0F8
:101F10000E941708609145018AE694E00E9406122B
:101F200062EC74E08AE694E00E941708CC2339F052
:101F30000E9409079091C8039111809345018AE698
:101F400094E00E94C2086DEA74E08AE694E00E9480
:101F50001708609146018AE694E00E9406126AEA38
:101F600074E08AE694E00E941708CC2339F00E94BE
:101F700009079091C8039111809346018AE694E085
:101F80000E94C20868E974E08AE694E00E9417089B
:101F90004091470150914801052E000C660B770BCC
:101FA0008AE694E00E94881165E974E08AE694E08C
:101FB0000E941708CC2359F00E9409079091C8038A
:101FC000992329F090E090934801809347018AE695
:101FD00094E00E94C20862E874E08AE694E00E94FD
:101FE0001708609149018AE694E00E9406126FE7A3
:101FF00074E08AE694E00E941708CC2339F00E942E
:1020000009079091C8039111809349018AE694E0F1
:102010000E94C20865E774E08AE694E00E9417080F
:1020200060914A018AE694E00E94061262E774E039
:102030008AE694E00E941708CC2339F00E94090731
:102040009091C803911180934A018AE694E00E941E
:10205000C208CC2329F00E94880ECF910C94690EFF
:10206000CF9108950E94071360E080E00E94BA11AA
:102070006CE674E082E495E00E94170865E674E07F
:1020800082E495E00E94170880919B02882339F032
:1020900060910B0182E495E00E94061206C063E69F
:1020A00074E082E495E00E94170862E080E00E94FC
:1020B000BA1180919A02882339F063EB73E082E4CD
:1020C00095E00E94D80806C065E574E082E495E0DA
:1020D0000E94170863E080E00E94BA116FE474E088
:1020E00082E495E00E94170868E371E082E495E0DD
:1020F0000E94D80864E080E00E94BA1169E474E0AC
:1021000082E495E00E94170880914201813019F421
:1021100061E474E002C069E374E082E495E00E9447
:10212000170865E080E00E94BA1163E374E082E47E
:1021300095E00E94170880914301813019F46BE209
:1021400074E002C062E274E082E495E00C94170847
:102150000E94071360E080E00E94BA1168E174E019
:1021600082E495E00E94170862E080E00E94BA11C4
:102170006CE074E082E495E00E94170863E080E080
:102180000E94BA1160E074E082E495E00E941708B2
:1021900042E050E060E070E082E495E00E94881147
:1021A0006EEF73E082E495E00E94170845E050E08E
:1021B00060E070E082E495E00C9488110E94D817EA
:1021C00084E98093BC008091BC0084FDFCCF80E05A
:1021D0000895CF938093BB000E94D81784E8809322
:1021E000BC008091BC0087FFFCCF8091B900887F44
:1021F000883299F08091B900C82FC87F8091B900CA
:10220000887F803319F40E94DE1005C01092BC0054
:1022100084E48093BC008C2F01C080E0CF910895AE
:10222000CF938093BB000E94D81784E88093BC00B2
:102230008091BC0087FFFCCF8091B900887F8831F6
:1022400029F08091B900887F803411F480E017C0B4
:102250008091B900C82FC87F8091B900887F8032F3
:1022600029F08091B900887F883419F40E94DE102B
:1022700005C01092BC0084E48093BC008C2FCF91E9
:1022800008950E94D81784EA8093BC008091BC0016
:1022900087FFFCCF8091B900887F883029F080913A
:1022A000B900887F803111F480E008958091B900F1
:1022B000887F883341F48091B9001092BC0094E487
:1022C0009093BC0002C08091B900887F0895CF939D
:1022D000C82F0E94D817CC2311F084EC01C084E8E9
:1022E0008093BC008091BC0087FFFCCF8091B90037
:1022F000887F883341F48091B9001092BC0094E447
:102300009093BC0002C08091B900887FCF9108955E
:10231000CF92DF92EF92FF920F931F93CF93DF93B1
:1023200077FF1DC06A017B01EC016DE20E9410087D
:102330008C0144275527BA014C195D096E097F09A4
:102340002AE0CE010E947908800F911FDF91CF9182
:102350001F910F91FF90EF90DF90CF9008952AE0AA
:10236000DF91CF911F910F91FF90EF90DF90CF9071
:102370000C947908CF93DF93262FC2E4D5E06A85C9
:102380000E949B24492F9C87822F90E02B8569E334
:10239000269F612D1124669570E06F5F7F4F0E942C
:1023A000A7248D87406860E0CE010E9432094D85E8
:1023B000406460E0CE01DF91CF910C9432090F931D
:1023C0001F93CF93DF93EC01AB01770F660B770B75
:1023D0000E9488118C01CE010E94C208800F911FBB
:1023E000DF91CF911F910F910895CF93DF93BC019F
:1023F0008AE694E00E946408EC018AE694E00E9478
:10240000C2088C0F9D1FDF91CF910895462F50E099
:1024100060E070E02AE00C9479081F93CF93DF937B
:10242000182FD62FC42F109248040E944111809378
:102430004804811127C0812F880F0E9410118093BA
:102440004804882321F08130E9F482E01BC08D2FFD
:102450000E94E91080934804882321F0813091F490
:1024600083E010C08C2F0E94E910809348048111F2
:10247000F5CF0E94DE1080934804882319F0813044
:1024800009F487E0DF91CF911F910895CF93DF93F7
:10249000D82FC09192051092950510929405109234
:1024A0004904109248040E9441118093480481110C
:1024B0003CC0CC0F8C2F0E941011809348048111D6
:1024C00034C08D2F0E94E9108093480481112DC0E3
:1024D0000E94411180934804811127C081E08C0F34
:1024E0000E9410118093480481111FC080914904FB
:1024F000811114C00E946711809348048835A9F4A3
:102500008091BB0080934A0481E08093950580937D
:1025100093050E94DE108093480407C081E00E946A
:10252000671180934804803559F380919505E091B7
:102530009305E81BE0939405811103C01092940564
:1025400007C0815080939505F0E0E85BFB4F8281E6
:10255000DF91CF9108951F93CF93DF9300D0CDB734
:10256000DEB7182F4A8369830E9446126981962F2D
:10257000909589234A814623482B612F80919205AB
:102580000F900F90DF91CF911F910C940D1240E0AE
:1025900061E080E00E94AB1246E96DE38091920514
:1025A0000E940D1262E070E080E090E00E948617C9
:1025B00040E260E288E00E94AB1262E070E080E0FE
:1025C00090E00E94861740E060E288E00C94AB1235
:1025D000893710F04FE007C0482F50E083E0559551
:1025E00047958A95E1F76FE088E00E94AB1261E1C0
:1025F00072E08AE694E00E94D80888E00E944612C1
:102600008F70682F70E08AE694E00C94DF11CF930E
:10261000DF9360E080E00E94BA11C0E0D0E09091CA
:102620004C0580914D05869586958695989FC001AD
:102630001124C817D90740F440E061E082E495E036
:102640000E9432092196EBCF60E080E0DF91CF91CC
:102650000C94BA11CF93DF93482F50E060E070E004
:102660002AE08AE694E00E947908EC018AE694E088
:102670000E94C2088C0F9D1FDF91CF910895CF92C9
:10268000DF92EF92FF92CF93DF9365EA79E08AE6DB
:1026900094E00E94C6081092C8030E94D817C0E0B8
:1026A000D0E06B017C0124EFC20E21E0D21EE11CC0
:1026B000F11C0E94D8176C157D058E059F0598F4B6
:1026C00083E295E00E94B306892B99F3CD37D105BB
:1026D00081F383E295E00E94CB06FE01E853FC4FB4
:1026E00080832196EDCFFE01E853FC4F1082CD2B65
:1026F00009F430C188EC93E00E94F5116EE979E0AD
:102700008AE694E00E94C60867E272E088EC93E0F3
:102710000E941025892B09F4AAC06EE879E08AE6A8
:1027200094E00E9417088AE694E00E94C208809113
:102730004B019091C7034091C6035091C50360E0DF
:1027400070E020E030E0F901E853FC4FE081EA332B
:1027500039F46115710521F42F5F3F4F61E070E09E
:10276000F901E853FC4FA081AA3379F56130710576
:1027700061F56281633539F463816537D9F4648129
:102780006E36C1F416C06D3439F463816F36C9F406
:1027900064816E36B1F4B9C0643509F0C2C063819A
:1027A000653709F0B4C06481653609F0B0C083E0D4
:1027B000AEC081E06381613621F46481643709F43D
:1027C00087E02F5F3F4F62E070E0F901E853FC4F74
:1027D000A081AA3379F56230710561F5DF011197A7
:1027E0009C91905311974C91440F4056542F550F84
:1027F000550F450F940F2F5F3F4F428160ED640FDF
:10280000D901A853BC4F5C91550F5056452F440F2A
:10281000440F540F462F450F558170ED750F64819D
:10282000660F6056562F550F550F650F572F560FD1
:1028300063E070E02F5F3F4F203831050CF483CF09
:1028400080934B014093C6035093C50320914701E9
:10285000920F983118F49093C70309C09851909340
:10286000C7038F5F883008F081E080934B016DE2F1
:1028700072E088EC93E00E941025892B09F46AC06D
:1028800066E879E08AE694E00E94170860E070E06C
:102890008AE694E00E94DF1188EC93E00E94F51133
:1028A000E8ECF3E0C0E0D0E060E070E080E090E0D1
:1028B0002191211106C0CE01861B970B409794F001
:1028C00049C08D379105B9F3223251F46115710574
:1028D00021F4209729F4BC0103C0209709F4EC01EE
:1028E0000196E6CF6C177D07ACF5CB0180959095EE
:1028F000C80FD91F67537C4FAE0183EB93E00E9452
:10290000FC24CD54DC4F188225C082E05ACF63816D
:10291000683609F056CF6481653709F052CF85E0FB
:1029200050CF673551F46381653609F04ACF648131
:10293000643609F046CF84E044CF663409F041CFD5
:102940006381623709F03DCF6481693609F039CF80
:1029500086E037CFDF91CF91FF90EF90DF90CF905F
:1029600008958F929F92AF92BF92EF92FF920F9332
:102970001F93CF93DF938C01892B11F401E819E0A9
:10298000C8010E946D24D82F80910D0590910E05ED
:10299000009751F020912205222331F06BE779E076
:1029A0000E941708109222050E94D8174B015C0163
:1029B000C0E080910B0590910C05DC01ED91FC913C
:1029C0000284F385E02D09957C011816190604F59B
:1029D00080910D0590910E05009741F0DC01ED917D
:1029E000FC910190F081E02D6E2D0995F801EC0F1E
:1029F000F11DE491F0E0EE16FF0621F4CF5FCD1358
:102A000002C01EC0C0E00E94D8174B015C01D1CFAC
:102A10000E94D817AB01BC01481959096A097B0902
:102A200080910F0590911005A0911105B0911205AC
:102A300084179507A607B70708F0BBCFC0E001C011
:102A4000C1E080910B0590910C05DC01ED91FC91AA
:102A50000084F185E02D0995892B61F080910B05AB
:102A600090910C05DC01ED91FC910680F781E02D41
:102A70000995E7CF80910D0590910E050E94C2083F
:102A80008C2FDF91CF911F910F91FF90EF90BF900E
:102A9000AF909F908F900895CF93DF93EC016FE6F6
:102AA00079E087E095E00E941708AE0160E070E0F1
:102AB0002AE087E095E00E94790887E095E00E948F
:102AC000C20880E090E0DF91CF910C94B11463E6EE
:102AD00079E087E095E00E94C6088AE599E00C94C9
:102AE000B114833081F028F4813099F08230A1F064
:102AF00008958730A9F08830B9F08430D1F48091FE
:102B000080008F7D03C0809180008F77809380004C
:102B1000089584B58F7702C084B58F7D84BD0895F4
:102B20008091B0008F7703C08091B0008F7D80933B
:102B3000B00008953FB7F89480919D0590919E054F
:102B4000A0919F05B091A00526B5A89B05C02F3F79
:102B500019F00196A11DB11D3FBFBA2FA92F982FC3
:102B60008827820F911DA11DB11DBC01CD0142E03E
:102B7000660F771F881F991F4A95D1F70895CF9246
:102B8000DF92EF92FF92CF93DF93EC0161E17AE065
:102B900087E095E00E941708BE0187E095E00E945B
:102BA00017086EE07AE087E095E00E94170860E57C
:102BB00070E087E095E00E94DF11C0900F05D09093
:102BC0001005E0901105F090120580911705909185
:102BD0001805A0911905B0911A050097A105B10536
:102BE00041F080930F0590931005A0931105B093C9
:102BF000120588E893E1A0E0B0E08093130590937C
:102C00001405A0931505B093160588E99AE3A0E092
:102C1000B0E08093170590931805A0931905B09321
:102C20001A0580E090E00E94B114C114D104E104BF
:102C3000F10441F0C0920F05D0921005E092110509
:102C4000F092120548E853E160E070E0409313050C
:102C500050931405609315057093160548E95AE3DF
:102C600060E070E0409317055093180560931905D4
:102C700070931A05882331F0D0932105C093200565
:102C800081E001C080E0DF91CF91FF90EF90DF9075
:102C9000CF90089580E480937C0080917A008064D6
:102CA00080937A0080917A0086FDFCCF8091780035
:102CB0002091790090E0922B0895CF92DF92EF92CD
:102CC000FF9263E372E08AE694E00E94D80880E015
:102CD0000E9446120E942A136EE372E08AE694E094
:102CE0000E94D80881E00E9446120E942A1369E4DB
:102CF00072E08AE694E00E94D80882E00E944612C0
:102D00000E942A1364E572E08AE694E00E94D808E3
:102D100083E00E9446120E942A136FE572E08AE661
:102D200094E00E94D80884E00E9446120E942A1370
:102D30006AE672E08AE694E00E94D80885E00E9484
:102D400046120E942A1365E772E08AE694E00E9428
:102D5000D80886E00E9446120E942A1360E872E0BA
:102D60008AE694E00E94D80887E00E9446120E94FA
:102D70002A136BE872E08AE694E00E94D80888E0A3
:102D80000E9446120E942A1386E00E9446128F710A
:102D9000C82ED12CDC2CCC240D2C000CEE08FF0806
:102DA00085E00E944612C82A84E00E944612FE2C4A
:102DB000ED2CDC2CCC24C82A66E07AE08AE694E08C
:102DC0000E9417082AE0B701A6018AE694E00E9453
:102DD00079088AE694E0FF90EF90DF90CF900C9412
:102DE000C208CF93DF93282F30E0F901EE50F64F61
:102DF0008491F901EC52F64FD491F901E054F64F69
:102E0000C491CC2391F081110E947115EC2FF0E058
:102E1000EE0FFF1FEA54F64FA591B491EC91ED230C
:102E200081E090E021F480E002C080E090E0DF915A
:102E3000CF9108951F93CF93DF93282F30E0F901AE
:102E4000EE50F64F8491F901EC52F64FD491F9010E
:102E5000E054F64FC491CC23C9F0162F81110E9483
:102E60007115EC2FF0E0EE0FFF1FE455F64FA59122
:102E7000B4918FB7F894111105C09C91ED2FE09596
:102E8000E92302C0EC91ED2BEC938FBFDF91CF9142
:102E90001F910895CF93DF9390E0FC01EC52F64F21
:102EA0002491FC01E054F64F8491882361F190E075
:102EB000880F991FFC01E851F64FC591D491FC0190
:102EC000E455F64FA591B491611109C09FB7F894EC
:102ED0008881209582238883EC912E230BC0623059
:102EE00061F49FB7F8943881822F8095832388837B
:102EF000EC912E2B2C939FBF06C08FB7F894E881DE
:102F00002E2B28838FBFDF91CF9108958F929F92B0
:102F1000AF92BF92CF92DF92EF92FF926B017C0152
:102F20000E949A154B015C01C114D104E104F10423
:102F3000F1F00E949A15DC01CB0188199909AA09C0
:102F4000BB09883E9340A105B10570F321E0C21A88
:102F5000D108E108F10888EE880E83E0981EA11CD4
:102F6000B11CC114D104E104F10419F7DDCFFF90C5
:102F7000EF90DF90CF90BF90AF909F908F9008958B
:102F80006AE070E080E090E00E94861783E00E9493
:102F900046128F70883031F0843031F0813031F05A
:102FA00080E0089581E0089582E0089583E0089527
:102FB0002FB7F8946091990570919A0580919B05BF
:102FC00090919C052FBF08951F920F920FB60F92FC
:102FD00011242F933F938F939F93AF93BF9380912F
:102FE000990590919A05A0919B05B0919C0530910F
:102FF000980523E0230F2D3720F40196A11DB11D64
:1030000005C026E8230F0296A11DB11D2093980547
:103010008093990590939A05A0939B05B0939C0586
:1030200080919D0590919E05A0919F05B091A0056E
:103030000196A11DB11D80939D0590939E05A093BF
:103040009F05B093A005BF91AF919F918F913F9144
:103050002F910F900FBE0F901F901895789484B504
:10306000826084BD84B5816084BD85B5826085BD84
:1030700085B5816085BD80916E00816080936E0012
:103080001092810080918100826080938100809104
:1030900081008160809381008091800081608093B5
:1030A00080008091B10084608093B1008091B00075
:1030B00081608093B00080917A00846080937A0070
:1030C00080917A00826080937A0080917A0081609A
:1030D00080937A0080917A00806880937A001092C1
:1030E000C10014BE61E08DE00E944A1761E084E0F7
:1030F0000E944A1760E082E00E944A1761E08CE07B
:103100000E944A1761E087E00E944A1761E08AE066
:103110000E944A1761E089E00E944A1761E08BE053
:103120000E944A1760E084E00E941A1760E08DE078
:103130000E941A17E0917A04F0917B0482E0808368
:10314000E0917604F09177041082E0917804F09198
:10315000790480E1808310928204E0917E04F091F2
:103160007F0486E08083E0917C04F0917D0480817F
:1031700080618083E0917C04F0917D04808188608F
:103180008083E0917C04F0917D048081806880835D
:10319000E0917C04F0917D0480818F7D808363E8E1
:1031A00071E08AE694E00E94170842E050E060E097
:1031B00070E08AE694E00E94881161E871E08AE696
:1031C00094E00E94170865E070E08AE694E00E94AF
:1031D000DF1164E671E08AE694E00E94C60866E5C5
:1031E00071E08AE694E00E94C60880E090E00E94C8
:1031F0007E0A90910C018913DDC30E944A16843F18
:1032000091400CF4D7C30E94690E80E090E00E94C8
:103210007E0A90910C01891709F46BC08AE694E04C
:103220000E94C20880E00E949F0E90914A0184E5AE
:1032300080934C0580E380934D0581E0913009F047
:1032400080E080934B0510924E0510924F0580E46C
:10325000E0E5F5E0DF011D928A95E9F761E08091F4
:1032600046050E944A1761E0809147050E944A176F
:1032700061E0809148050E944A1761E0809149050C
:103280000E944A1761E080914A050E944A1761E056
:10329000809149050E941A1761E080914A050E94B9
:1032A0001A1760E0809149050E941A1764E670E0E1
:1032B00080E090E00E94861761E0809149050E94BD
:1032C0001A1741E260E082E495E00E94320943E18E
:1032D00060E082E495E00E94320980914B058130E4
:1032E000B9F440EE60E082E495E00E94320945E0E6
:1032F00010C0C0E0D0E0CE010E947E0A682F8AE6AE
:1033000094E00E94D3052196CF33D105A1F786CF53
:1033100042EC60E082E495E00E94320940E260E025
:1033200082E495E00E94320949E060E082E495E0A1
:103330000E9432090E94071348E060E082E495E0B1
:103340000E9432094CE060E082E495E00E9432097C
:1033500064E670E080E090E00E94861740E860E05C
:1033600082E495E00E94320940E460E082E495E066
:103370000E94320968EC70E080E090E00E948617BD
:103380000E94A81068EE73E080E090E00E9486172B
:1033900010923E0510923D0510923C0510923B059F
:1033A00010923A05109239058DE991E0909340050D
:1033B00080933F0590912F05963108F057C02DEB73
:1033C00030E030933A05209339052BE931E0309312
:1033D0003C0520933B052CE231E030933E052093E1
:1033E0003D0520916800983050F031E09E3008F49F
:1033F00030E081E001C0880F3A95EAF701C084E02F
:10340000822B80936800983038F09E3040F09631DF
:1034100048F020E030E008C02DE630E005C02BE6A3
:1034200030E002C02CE630E03093370520933605BB
:10343000983030F481E001C0880F9A95EAF70EC009
:10344000292F30E09E3018F42850310902C02E5048
:10345000310981E001C0880F2A95EAF78093380589
:1034600080913F05909140050197F1F780913D05CE
:1034700090913E05892B21F18091980290919902BB
:10348000B5E083329B07E1F0009711F00E945E0ADD
:10349000809141058E7F8093410510929702109292
:1034A000960283E295E09093990280939802E091CE
:1034B0003605F0913705908180913805892B8083FE
:1034C00069E271E08AE694E00E94C60868E873E168
:1034D00080E090E00E9486178AE694E00E949C05B6
:1034E000892B09F46FC069E171E08AE694E00E94DB
:1034F000C608E0E0F1E001900020E9F73197EF0124
:10350000C050D14009F44FC000E010E08AE694E0DA
:103510000E94E00797FD56C0F801E050FF4F208160
:10352000022E000C330B82179307B9F10115110518
:1035300021F420E030E08901E9CF9801A901415050
:103540005109FA01E050FF4F6081062E000C770B05
:1035500086179707F1F44115510569F3A0E0B1E032
:1035600060E070E07801E41AF50ADD90FB01EE0DF1
:10357000FF1DE050FF4FE081DE1629F0641775074C
:10358000D1F29A01DBCF6F5F7F4F6417750768F345
:10359000F5CF41155105A9F7CCCF98012F5F3F4FCB
:1035A0002C173D0741F668E071E08AE694E00E943E
:1035B000C60881E00E949F0E60ED77E080E090E019
:1035C0000E948617449A459A8091B9008E7F809315
:1035D000B9008091B9008D7F8093B90088E4809311
:1035E000B80084E48093BC00449A459A8CE08093B0
:1035F000B80062E070E080E090E00E94861746E943
:103600006CE3809192050E940D1262E070E080E010
:1036100090E00E948617D091430110914201C09121
:1036200045010E94C712113041F44CE16EE380E085
:103630000E94AB1284E991E007C044E26EE380E0AF
:103640000E94AB1281EB91E00E94F511D11106C0EE
:1036500040E260E283E00E94AB1209C040E060E219
:1036600083E00E94AB128DEC91E00E94F51140E0E6
:1036700060EE88E00E94AB1264EF71E080E090E0C1
:103680000E9486178C2F0E94E81289EE91E00E941A
:10369000F51140914601483018F44295407F01C031
:1036A00040E260E781E00E94AB126AE070E080E0F7
:1036B00090E00E948617F89414BE809160008861A3
:1036C0008093600081E680936000109280001092E9
:1036D00081008EEE95E89093850080938400809120
:1036E000810084608093810080916F00816080936D
:1036F0006F0078940E945D1610929E026AE070E05E
:1037000080E090E00E9486170E94A81068EE73E0A7
:1037100080E090E00E94861768EF70E08AE694E00F
:103720000E941708C0E0D0E0FE01E755FD4F10826F
:10373000118212821382148266EF70E08AE694E0AE
:103740000E9417082596C233D10571F78AE694E0E6
:103750000E94C20864EE70E08AE694E00E94C60807
:103760000E94071362E370E080E090E00E948617F9
:103770008AE694E00E94C208B12C00E010E0C0E0AC
:10378000D0E0E7EEEE2EE3E0FE2E702E40E060EC9F
:1037900083E00E94AB1240E860EE88E00E94AB122A
:1037A0008B2D0E94E81269E170E080E090E00E94B9
:1037B0008617809190050E94F1164C010E94D8173F
:1037C0001B012C01E4E62E0E311C411C511CC12CA6
:1037D000D12C0E94D817DC01CB0182199309A409CE
:1037E000B509B7FF0CC0809190050E94F1168816AC
:1037F00099061CF4FFEFCF1ADF0A4C01EACF62E012
:1038000070E080E090E00E94861740E060EE88E083
:103810000E94AB120E94C712AC2CDD24CE14DF0430
:1038200014F4E801760169EC70E08AE694E00E9405
:103830001708672D8AE694E00E94061265EB70E097
:103840008AE694E00E941708A601DD0C660B770B50
:103850008AE694E00E94881164E072E08AE694E0CF
:103860000E94D8082A2D30E0A0EAB0E00E948C2403
:10387000AB01BC018AE694E00E94881188E092E0E6
:103880000E94F51164E170E080E090E00E948617EC
:103890000F5F1F4F28E0B20E30E8B31276CF67EA11
:1038A00070E08AE694E00E941708AE010D2E000C2D
:1038B000660B770B8AE694E00E9488116CE970E051
:1038C0008AE694E00E94170863E0CC0FDD1F6A953A
:1038D000E1F7BE018AE694E00E94DF1160E080E03B
:1038E0000E94BA1162E970E082E495E00E94170834
:1038F000AE01DD0F660B770B82E495E00E94881124
:103900000E94800A0E944A1690936A03809369037A
:103910000E9407130E94321070EF272E76E0372E98
:103920000FE315E080919F0281111DC069EC71E0E9
:1039300087E095E00E9417082AE040E050E0BA01D5
:1039400087E095E00E94790887E095E00E94C20830
:1039500062EC71E080910D0590910E050E94C60801
:1039600081E080939F0230920401209203018091B4
:103970006900836080936900E89A0E94C0171092E2
:103980009E0283E080937103BB24B39480919E02D6
:1039900081113EC00E944A16853F9140CCF1909122
:1039A000C60380916B03981333C080916C0381111F
:1039B0002FC009C061E471E08AE694E00E94C60865
:1039C0000E94880E20CCC0906D03D0906E03E090D2
:1039D0006F03F0907003C114D104E104F104B1F25B
:1039E0000E94D817DC01CB018C199D09AE09BF09D3
:1039F00081319742A105B10548F2B0926C03109253
:103A00006D0310926E0310926F0310927003BECF7D
:103A1000A89510929D0210929C0210926C0361E096
:103A20008DE00E941A1744E260E082E495E00E9473
:103A3000320980919E0218161CF482E08093710373
:103A400065E070E080E090E00E948617E8981093AF
:103A50000401009303010E944A1690936A03809325
:103A600069039091C60380916B03891709F482C0A2
:103A700080910B018F5F80930B0190936B031092E9
:103A8000710380916803811175C0A4E6B3E0C5E6B7
:103A9000D3E0E9E2F3E02E912A9323E0A932B207C2
:103AA000D1F71092290380E09191891708F4892FAA
:103AB00033E0E536F307C1F78093A0026EE10E9480
:103AC0009B24811101C081E0809307011092A40220
:103AD0008091C70390916703891719F18093670359
:103AE000A0E1B3E0C1E1D3E0E9EFF2E02E912A9347
:103AF00042E0A93FB407D1F71092F90280E091911A
:103B0000891708F4892F93E0E131F907C1F7809311
:103B1000A1026EE10E949B24811101C081E080938B
:103B2000080180914B0190910A01891719F1809346
:103B30000A01A8EFB2E0C9EFD2E0EBEDF2E02E917E
:103B40002A9322E0AB3DB207D1F71092DB0280E06E
:103B50009191891708F4892F32E0E93FF307C1F703
:103B60008093A2026EE10E949B24811101C081E03A
:103B70008093090180916603882329F010926603DF
:103B80008CE380930B0180910B018C3399F410929C
:103B90009B0210920B010E94800A80919A02882356
:103BA00049F081E080939B020E942F0D60E080E04D
:103BB0000E945D0DE0906903F0906A0344EFE41603
:103BC00041E0F4060CF027C1C1E0C09371030E94EC
:103BD000740A68EC70E080E090E00E94861780E94B
:103BE000E81681E0F8060CF034C59CE2E91691E095
:103BF000F9061CF0C093A3020FC0A8ECEA16F1046A
:103C000014F082E007C0B2E3EB16F10414F083E095
:103C100001C084E08093A30262EE71E08AE694E042
:103C20000E941708809149010E942A1362ED71E0F9
:103C30008AE694E00E9417088091A3020E942A134A
:103C40002091A30230E0F89480914901823081F400
:103C500090916503992361F091E09093680324307B
:103C6000310509F0A2C09091650391110AC043C0CB
:103C7000109268032430310509F048C08230D9F52C
:103C8000F2CF913031F480914B018F5F80934B01E3
:103C900017C0923031F48091C7038F5F8093C703C0
:103CA0000FC0933031F48091C6038F5F8093C603B9
:103CB00007C0943029F48091C5038F5F8093C503BA
:103CC00080914B01883018F081E080934B01809106
:103CD000C703883110F01092C7038091C6038C335C
:103CE00010F01092C6038091C5038C3308F47DC098
:103CF0001092C5037AC08F5F853018F48093490114
:103D000002C010924901109265036FC02230310544
:103D100009F04FC0823009F041C0909165039923AA
:103D2000E9F1913031F480914B01815080934B0146
:103D300017C0923031F48091C70381508093C7033C
:103D40000FC0933031F48091C60381508093C60335
:103D500007C0943029F48091C50381508093C50336
:103D600080914B01883018F087E080934B0180915F
:103D7000C703883118F087E18093C7038091C60399
:103D80008C3318F08BE38093C6038091C5038C338A
:103D900008F440C08BE38093C5033CC0815085305C
:103DA00008F084E08093490133C02230310509F4E2
:103DB000B4CF23303105C9F49091650391509093AD
:103DC0006503813021F4933028F182E005C0823010
:103DD00031F49530F8F084E0809365031BC08111C5
:103DE00019C081E08093660315C02130310591F43C
:103DF000809165038F5F80936503909149019130B5
:103E000019F4833038F004C0923021F4853010F07A
:103E10001092650378946BEE73E08AE694E00E945A
:103E20001708609171038AE694E00E9406126DED16
:103E300073E08AE694E00E94170840916D03509168
:103E40006E0360916F03709170032AE08AE694E03C
:103E50000E9479088AE694E00E94C208809171036A
:103E6000833008F0F3C3823009F0E7C10E94740A7E
:103E7000E0914B018E2F90E0FC013197E730F10586
:103E8000E0F4EC5CFF4F0C94DD246DE172E011C0B6
:103E900066E172E00EC06EE072E00BC064E072E0BA
:103EA00008C06BEF71E005C064EF71E002C06BEE1B
:103EB00071E08AE694E00E94170860E28AE694E0E6
:103EC0000E9410088091C7038A3028F460E38AE6D4
:103ED00094E00E9410086091C7038AE694E00E9473
:103EE00006126AE38AE694E00E9410088091C603F5
:103EF0008A3028F460E38AE694E00E94100860911A
:103F0000C6038AE694E00E9406126AE38AE694E019
:103F10000E9410088091C5038A3028F460E38AE685
:103F200094E00E9410086091C5038AE694E00E9424
:103F3000061260E28AE694E00E9410080E940713CD
:103F40000E94C01710929E02811123C06BEF72E095
:103F50008AE694E00E94C6080E94071360E080E0B1
:103F60000E94BA1161EF72E082E495E00E941708A6
:103F700061E080E00E94BA1162EE72E082E495E0B6
:103F80000E94170862E080E00E94BA1164ED72E0BE
:103F900034C1813009F0EFC087E00E944612C82F7B
:103FA000CF736BEA72E08AE694E00E9417086C2FE8
:103FB0008AE694E00E9406126FE972E08AE694E0D5
:103FC0000E94C6080E94071360E080E00E94BA11B8
:103FD00065E972E082E495E00E94170861E080E004
:103FE0000E94BA116CE872E082E495E00E94170822
:103FF0006C2F82E495E00E94061268E872E082E489
:1040000095E00E9417088091A7029091A80201965E
:104010009093A8028093A702809129038F5F8093D9
:1040200029038091F9028F5F8093F9028091DB026E
:104030008F5F8093DB02A6EDB2E025E0CD0105970E
:10404000FC01322F01900D923A95E1F7DC01895A7B
:104050009240A1F780914B018093A9028091C70300
:104060008093AA028091C6038093AB028091C5031E
:104070008093AC02C093AD026C2F81E00E945D0D75
:1040800010920B01C12CD12CE601C755DD4F688180
:104090008AE694E00E94061266E872E08AE694E0FE
:1040A0000E94170869818AE694E00E94061264E87B
:1040B00072E08AE694E00E9417086A818AE694E03A
:1040C0000E94061262E872E08AE694E00E941708F5
:1040D0006B818AE694E00E9406126BE772E08AE642
:1040E00094E00E9417086C818AE694E00E94061210
:1040F00067E772E08AE694E00E94C608F5E0CF0E1A
:10410000D11C22E3C216D10409F0BECF8091440134
:10411000882331F190912903981710F18091A4021E
:1041200081111EC055E0E52EF12C61E084E00E9473
:104130001A1768EC70E080E090E00E94861760E05B
:1041400084E00E941A1768EC70E080E090E00E9422
:10415000861731E0E31AF10841F781E08093A40269
:104160000E94D81760936D0370936E0380936F0362
:104170009093700346C0823031F564E672E08AE6BF
:1041800094E00E94C6080E94071360E080E00E944D
:10419000BA116AE572E082E495E00E94170861E0D6
:1041A00080E00E94BA116FE472E082E495E00E9420
:1041B00017088091A5029091A60201969093A602FD
:1041C0008093A5021EC08330E1F40E94071360E0D3
:1041D00080E00E94BA116AE372E08AE694E00E94ED
:1041E000C6086EE272E082E495E00E94170861E082
:1041F00080E00E94BA1164E272E082E495E00E94DD
:1042000017080E945D164FE16FE187E00E94AB1234
:1042100040E460E482E00E94AB1240E060E482E0AF
:104220000E94AB1240E460E482E00E94AB1264EFB3
:1042300071E080E090E00E94861780914901811131
:1042400062C00E94071360E080E00E94BA1162E43D
:1042500073E082E495E00E94170862E080E00E942B
:10426000BA116AE373E082E495E00E941708609156
:10427000290382E495E00E94061263E080E00E9438
:10428000BA1162E373E082E495E00E94170860913E
:10429000F90282E495E00E94061264E080E00E9448
:1042A000BA116AE273E082E495E00E941708609117
:1042B000DB0282E495E00E94061265E080E00E9445
:1042C000BA1162E273E082E495E00E94170840911F
:1042D000A7025091A80260E070E02AE082E495E035
:1042E0000E94790860E273E082E495E00E9417087A
:1042F0004091A5025091A60260E070E02AE082E4BD
:1043000095E00E94790880914901813031F08091D7
:104310004901823009F084C1B5C00E94071360E0F2
:1043200080E00E94BA116EE673E082E495E00E949C
:10433000170880916503823021F044E0A42EB12C4F
:1043400003C032E0A32EB12C9DEAC92E92E0D92EF3
:10435000E12CF12C25E0822E80916503D701E4E069
:104360008E9FA00DB11D11248A9EF0018B9EF00D31
:104370001124E755FD4F72806180508082E0982EB5
:104380009E0C692D80E00E94BA11852D90E0FC0101
:104390003197E730F105C8F4E55CFF4F0C94DD245C
:1043A00065E673E014C061E673E011C06DE573E08B
:1043B0000EC069E573E00BC065E573E008C061E518
:1043C00073E005C06DE473E002C069E473E082E469
:1043D00095E00E941708692D85E10E94BA11F9E065
:1043E000F61528F060E382E495E00E941008662D3F
:1043F00082E495E00E9406126AE382E495E00E945E
:10440000100829E0271528F060E382E495E00E9477
:104410001008672D82E495E00E940612692D89E359
:104420000E94BA11D6018C918A3030F46CE673E0A8
:1044300082E495E00E94170880916503F70124E06B
:10444000829FE00DF11D1124CF01889EF001899E0D
:10445000F00D1124E755FD4F648182E495E00E9440
:10446000061269E673E082E495E00E9417083FEFC8
:10447000E31AF30A45E0C40ED11CEA14FB0409F068
:104480006BCF45CF0E94071361E080E00E94BA1114
:104490008091C7038A3028F460E382E495E00E94AB
:1044A00010086091C70382E495E00E9406126AE357
:1044B00082E495E00E9410088091C6038A3028F4B7
:1044C00060E382E495E00E9410086091C60382E4F4
:1044D00095E00E9406126AE382E495E00E941008CB
:1044E0008091C5038A3028F460E382E495E00E945D
:1044F00010086091C50382E495E00E940612809145
:104500006503823051F460E080E00E94BA116AEDE8
:1045100073E082E495E00E94170880916503833080
:1045200051F460E080E00E94BA1164ED73E082E42F
:1045300095E00E94170880916503843051F460E093
:1045400080E00E94BA116BEC73E082E495E00E9477
:10455000170860E080E00E94BA1180916503823004
:1045600078F5E0914B018E2F90E0FC013197E73018
:10457000F105E0F4EE5BFF4F0C94DD2464EC73E096
:1045800011C06DEB73E00EC065EB73E00BC06BEA1E
:1045900073E008C062EA73E005C06BE973E002C033
:1045A00062E973E082E495E00E9417088091650358
:1045B000813031F46FE873E082E495E00E941708DF
:1045C00063E080E00E94BA1167E873E082E495E05E
:1045D0000E9417086091290382E495E00E94061268
:1045E00064E080E00E94BA116FE773E082E495E036
:1045F0000E9417086091F90282E495E00E94061279
:1046000065E080E00E94BA1167E773E082E495E01C
:104610000E9417086091DB0282E495E00E94061276
:1046200080914901833011F40E94A81080914901C2
:10463000843011F40E9432100E94D81760936D03E9
:1046400070936E0380936F03909370030E943C06F7
:1046500069C91092A302E0CA8EE691E09093240506
:104660008093230583E295E00C945E0ACF92DF925B
:10467000EF92FF92CF9310926D0410926C0498EE1B
:10468000C92E93E0D92EE12CF12CC0926E04D09269
:104690006F04E0927004F092710480E591E09093D1
:1046A0006B0480936A0485EC90E090937704809388
:1046B000760484EC90E0909379048093780480EC05
:1046C00090E090937B0480937A0481EC90E0909347
:1046D0007D0480937C0482EC90E090937F0480932F
:1046E0007E0486EC90E09093810480938004109285
:1046F000830410928404109285041092860480E54D
:10470000809396051092970583E080939205C9E007
:10471000C093910582E08093900561E089E00E945A
:104720004A1760E0809190050E944A1761E08091ED
:1047300091050E941A17109245051092440580E8D1
:1047400091E0909343058093420587E0809346056E
:104750008CE0809347058BE0809348058AE0809346
:104760004905C0934A051092260510922505C0926E
:104770002705D0922805E0922905F0922A058EE6B9
:1047800091E0909324058093230510923A051092AE
:10479000390510923C0510923B0510923E0510928F
:1047A0003D051092400510923F05609141056E7FD6
:1047B0006D7F609341056695617081E0682783E0B5
:1047C0000E941A1761E083E00E944A17E7EDF9E0C2
:1047D000E491E0933305E3ECF9E0E491F0E0EE0FCF
:1047E000FF1FE455F64F8591949190933505809382
:1047F000340560E085E00E944A178091410581FD03
:1048000004C061E085E00E941A1785E080932F05BF
:10481000E9EDF9E0E491E0933005E5ECF9E0E491AD
:10482000F0E0EE0FFF1FEA54F64F859194919093BC
:1048300032058093310510920A051092090582E62F
:1048400091E0909308058093070583E295E09093AB
:104850000C0580930B058AE694E090930E058093F7
:104860000D0586E080931F0510922105109220050A
:104870001092220588EE93E0A0E0B0E080930F054F
:1048800090931005A0931105B093120588E893E169
:10489000A0E0B0E08093130590931405A093150554
:1048A000B093160588E99AE3A0E0B0E0809317057D
:1048B00090931805A0931905B0931A05CF91FF9016
:1048C000EF90DF90CF900895FB01DC0102C00590CE
:1048D0000D9241505040D8F70895FC0105900020FA
:1048E000E9F7809590958E0F9F1F0895F999FECF57
:1048F00092BD81BDF89A992780B50895262FF99920
:10490000FECF1FBA92BD81BD20BD0FB6F894FA9AB2
:10491000F99A0FBE01960895A29FB001B39FC001FE
:10492000A39F700D811D1124911DB29F700D811DDB
:104930001124911D0895991B79E004C0991F9617C1
:1049400008F0961B881F7A95C9F78095089597FB04
:10495000072E16F4009407D077FD09D00E94E324B7
:1049600007FC05D03EF4909581959F4F0895709572
:1049700061957F4F0895A1E21A2EAA1BBB1BFD0172
:104980000DC0AA1FBB1FEE1FFF1FA217B307E4072E
:10499000F50720F0A21BB30BE40BF50B661F771F86
:1049A000881F991F1A9469F7609570958095909566
:1049B0009B01AC01BD01CF010895EE0FFF1F0590D3
:1049C000F491E02D0994AA1BBB1B51E107C0AA1F5B
:1049D000BB1FA617B70710F0A61BB70B881F991FA0
:1049E0005A95A9F780959095BC01CD01089581E075
:1049F00090E0F8940C942A25FB01DC0102C00190A0
:104A00000D9241505040D8F70895FB01DC010D9004
:104A10000020E9F7119701900D920020E1F7089529
:104A2000FB0151915523A9F0BF01DC014D914517C0
:104A30004111E1F759F4CD010190002049F04D9169
:104A400040154111C9F3FB014111EFCF81E090E026
:104A50000197089515E0C4E1D5E004C0FE010E946D
:0E4A6000DD242196C531D107C9F7F894FFCFA8
:104A6E004753003F053F050101010137404D4152BB
:104A7E004F44454B457874656E646572003039312C
:104A8E0039393332303033000000000000000000AE
:104A9E00000000000000000050413252444B000064
:104AAE00000001010270020100004201000000003E
:104ABE00D30540056B051A069C057A058E05000088
:104ACE0000003B084005ED06EC06000000005F0606
:104ADE004005ED065E06B306CB0646060000000056
:104AEE006B094005ED06EC0600000000900740053E
:104AFE00ED06EC0673657420757020666F72206F7C
:104B0E007574646F6F72206F7065726174696F6E09
:104B1E000073657420757020666F7220696E646F05
:104B2E006F72206F7065726174696F6E0064697365
:104B3E0074757262657220646574656374696F6EF4
:104B4E0020656E61626C65640041533339333520E4
:104B5E006D616E75616C2063616C20636F6D706C3E
:104B6E0065746500203D200020487A000D0A002E55
:104B7E000063617061636974616E6365207365744F
:104B8E0020746F20387800446174653A00535441A4
:104B9E0049500052656720307830303A2000526517
:104BAE006720307830313A200052656720307830F7
:104BBE00323A200052656720307830333A20005266
:104BCE00656720307830343A20005265672030789F
:104BDE0030353A200052656720307830363A200062
:104BEE0052656720307830373A20005265672030A2
:064BFE007830383A200077
:00000001FF
